:020000040800F2
:1000000000000120290200086D0200086D020008AE
:100010006D0200086D0200086D020008000000007B
:100020000000000000000000000000006D02000859
:100030006D020008000000006D0200086D0200085B
:100040006D0200086D0200086D0200086D020008D4
:100050006D0200086D0200086D0200086D020008C4
:100060006D0200086D0200086D0200086D020008B4
:100070006D0200086D0200086D0200086D020008A4
:100080006D0200086D0200086D0200086D02000894
:100090006D0200086D0200086D0200086D02000884
:1000A0006D0200086D0200086D0200086D02000874
:1000B0006D0200086D0200086D0200086D02000864
:1000C0006D0200086D0200086D0200086D02000854
:1000D0006D0200086D0200086D0200086D02000844
:1000E0006D0200086D0200086D0200086D02000834
:1000F0006D0200086D0200086D0200086D02000824
:100100006D0200086D0200086D0200086D02000813
:100110006D0200086D0200086D0200086D02000803
:100120006D0200086D0200086D0200086D020008F3
:1001300000000000000000000000000000000000BF
:1001400000000000000000000000000000000000AF
:10015000000000000000000000000000000000009F
:10016000000000000000000000000000000000008F
:10017000000000000000000000000000000000007F
:10018000000000000000000000000000000000006F
:10019000000000000000000000000000000000005F
:1001A000000000000000000000000000000000004F
:1001B000000000000000000000000000000000003F
:1001C000000000000000000000000000000000002F
:1001D000000000000000000000000000000000001F
:0401E0005FF8E0F1F3
:1001E40010B5054C237833B9044B13B10448AFF36D
:1001F40000800123237010BD0000002000000000D7
:10020400E401000808B5034B1BB103490348AFF3ED
:10021400008008BD0000000004000020E401000884
:10022400FEE70000002103E00A4B5B584350043111
:1002340009480A4B42189A42F6D3094A02E00023BD
:1002440042F8043B074B9A42F9D300F075F8FFF7E4
:10025400E7FF7047000000000000002000000020BD
:10026400000000201C000020FEE7000082B00023F4
:10027400019300932C4A136843F4803313602A4B90
:100284001B6803F400330093019B01330193009B2B
:100294001BB9019BB3F5A06FF1D1234B1B6813F479
:1002A400003F06D001230093009B012B04D002B031
:1002B400704700230093F7E71C4B1A6842F01002C2
:1002C4001A601A6822F007021A601A6842F00202E1
:1002D4001A60A3F580535A685A605A685A605A687B
:1002E40042F480625A605A6822F47C125A605A6856
:1002F40042F4E8125A601A6842F080721A600A4B9B
:100304001B6813F0007FFAD0074B5A6822F00302EF
:100314005A605A6842F002025A60034B5B6803F069
:100324000C03082BF9D1C2E7001002400020024060
:1003340008B5FFF79BFF08BD08B5104B1A6842F0DB
:1003440001021A6059680E4A0A405A601A6822F07B
:10035400847222F480321A601A6822F480221A60AD
:100364005A6822F4FE025A604FF41F029A60FFF7A3
:10037400DFFF044B4FF000629A6008BD001002409A
:100384000000FFF800ED00E0F8B500BFF8BC08BCC1
:100394009E467047F8B500BFF8BC08BC9E4670473F
:0403A4000902000842
:0403A800E501000863
:0400000508000229C4
:00000001FF
